:100000000C9442050C9489050C9489050C9489057F
:100010000C9489050C9489050C9489050C94890528
:100020000C9489050C9489050C9489050C940B0F8C
:100030000C94BA0F0C94CD1E0C9489050C94890570
:100040000C9489050C9489050C9489050C94411F26
:100050000C9489050C9489050C9489050C948905E8
:100060000C9489050C9489050C9489050C948905D8
:100070000C948905271049103711491037118E103B
:10008000B110371106111911E614E61415151515DE
:100090007315B115CB17CB17CA15CB17CB16CB16CB
:1000A0009F17CB17CB17B617041607090B0A1D1B92
:1000B00006196405141A08151C171E1F2021232277
:1000C0002E26242D25273012182F0C13280F0D341F
:1000D0000E333136381110372B2C352A5829787BBE
:1000E00079397A504F5152726C63685680668053EA
:1000F000020103555880576D6E5462595A5B5C5D1E
:100100005E5F6F60617475663E3F403C414277447C
:1001100076466B47804365458048494A4B4C3D4D88
:100120003B4E3A7D7E7C7F736164625F686F73745F
:100130005F6B62645F726563763A204552524F523C
:10014000282564290A000A002530345800616462B9
:100150005F686F73745F6B62645F726563763A2089
:10016000004552524F523A206D65646961206B65BB
:1001700079300A004552524F523A206D65646961E8
:10018000206B6579310A005D0A0025640020002596
:1001900064007C00253032580020002530325800A1
:1001A0006164625F6D6F757365207261773A205B81
:1001B000000A002530313662006164625F686F7347
:1001C000745F6D6F7573655F726563763A20006466
:1001D0006562756720656E61626C65642E0A005306
:1001E00063616E3A20616464723A25642C20726502
:1001F00067333A253034580A0041667465722069C5
:100200006E69743A0A00466F756E643A206D6564D3
:100210006961206B6579730A005363616E3A2061EE
:100220006464723A25642C20726567333A25303451
:10023000580A004265666F726520696E69743A0AF1
:10024000004B6579626F6172642073746172742E01
:100250000A0055534220636F6E6669677572656464
:100260002E0A000D0A696E69740A002E03410044CB
:1002700000420020006B006500790062006F0061A1
:100280000072006400200063006F006E007600655D
:1002900000720074006500720000000E0374002EEE
:1002A000006D002E006B002E0000000403090409FD
:1002B000027400040100A0320904000001030101DE
:1002C00000092111010001224000070581030800F7
:1002D0000A090401000103010200092111010001C2
:1002E000224D000705820308000A090402000103E9
:1002F00000000009211101000122360007058303D7
:1003000008000A090403000203000000092111018A
:1003100000012222000705840320000107050403D1
:100320002000011201100100000008EDFEDB0A01AF
:1003300001010200010631FF0974A10109751500D0
:1003400026FF009520750881020976150026FF001A
:10035000952075089102C005010980A1018502164A
:10036000810026B7001A81002AB700751095018117
:1003700000C0050C0901A1018503160100269C029D
:100380001A01002A9C02751095018100C00501091F
:1003900002A1010901A1000509190129051500257E
:1003A000019505750181029501750381010501091A
:1003B0003009311581257F950275088106093815A8
:1003C00081257F950175088106050C0A3802158183
:1003D000257F950175088106C0C005010906A101A8
:1003E000050719E029E71500250195087501810227
:1003F0009501750881010508190129059505750103
:1004000091029501750391010507190029FF150057
:1004100026FF00950675088100C0636F6E73756DC9
:1004200065723A20253034580A0073797374656D0B
:100430003A20253034580A000A002530325820006E
:100440006B6579626F6172643A20004C45443A20D2
:10045000253032580A00253032583A20253038628B
:1004600025730A00722F632030313233343536372A
:100470000A00290A002575002F002575005D280057
:10048000256400200025640020002564002000254C
:1004900064007C0025303258006D6F7573656B65A4
:1004A00079205B62746E7C782079207620685D28E4
:1004B0007265702F61636C293A205B006D6B5F770A
:1004C0006865656C5F74696D655F746F5F6D617899
:1004D000203D2025640A006D6B5F776865656C5F61
:1004E0006D61785F7370656564203D2025640A0046
:1004F0006D6B5F74696D655F746F5F6D6178203DD2
:100500002025640A006D6B5F6D61785F73706565AF
:1005100064203D2025640A006D6B5F696E7465720E
:1005200076616C203D2025640A006D6B5F64656C0C
:100530006179203D2025640A006D6B5F77686565F1
:100540006C5F74696D655F746F5F6D6178203D20CD
:1005500025640A006D6B5F776865656C5F6D617817
:100560005F7370656564203D2025640A006D6B5FD4
:1005700074696D655F746F5F6D6178203D202564DF
:100580000A006D6B5F6D61785F7370656564203D17
:100590002025640A006D6B5F696E74657276616C0C
:1005A000203D2025640A006D6B5F64656C617920D5
:1005B0003D2025640A000A00257500363A20776838
:1005C00065656C5F74696D655F746F5F6D61783AC6
:1005D00020000A00257500353A20776865656C5F54
:1005E0006D61785F73706565643A20000A00257557
:1005F00000343A2074696D655F746F5F6D61783A9D
:1006000020000A00257500333A206D61785F737011
:100610006565643A20000A00257500323A20696E4B
:1006200074657276616C286D73293A20000A002582
:100630007500313A2064656C6179282A31306D7318
:10064000293A20000A092D2056616C756573202D0A
:100650000A004D3E004D25643E20003F0073657446
:100660002064656661756C740A00433E20007768FB
:100670006572652064656C74613A20637572736F8E
:10068000723D25642C20776865656C3D25640A53AE
:10069000656520687474703A2F2F656E2E77696BCC
:1006A0006970656469612E6F72672F77696B692F56
:1006B0004D6F7573655F6B6579730A000A092D20AC
:1006C0004D6F7573656B6579202D0A4553432F7106
:1006D0003A09717569740A313A0964656C6179285F
:1006E0002A31306D73290A323A09696E746572765F
:1006F000616C286D73290A333A096D61785F7370F4
:100700006565640A343A0974696D655F746F5F6D7D
:1007100061780A353A09776865656C5F6D61785F65
:1007200073706565640A363A09776865656C5F744D
:10073000696D655F746F5F6D61780A0A703A097060
:1007400072696E742076616C7565730A643A097318
:1007500065742064656661756C74730A75703A0916
:100760002B310A646F776E3A092D310A7067757004
:100770003A092B31300A7067646F776E3A092D3170
:10078000300A0A7370656564203D2064656C74618D
:10079000202A206D61785F7370656564202A2028A7
:1007A000726570656174202F2074696D655F746F68
:1007B0005F6D6178290A003F004D3E2000433E20D6
:1007C000004C25640A000A092D20436F6E736F6C7C
:1007D00065202D0A4553432F713A09717569740AD2
:1007E0006D3A096D6F7573656B65790A000A092D9D
:1007F000204D61676963202D0A643A09646562755A
:10080000670A783A096465627567206D6174726978
:10081000780A6B3A096465627567206B6579626F67
:100820006172640A6D3A096465627567206D6F755F
:1008300073650A763A0976657273696F6E0A733A60
:10084000097374617475730A633A09636F6E736F29
:100850006C65206D6F64650A302D343A096C6179DE
:100860006572302D34284631302D4634290A5061C6
:1008700075733A09626F6F746C6F616465720A0018
:100880003F0074696D65725F726561643332282957
:100890003A202530346C580A006B6579626F6172BA
:1008A000645F69646C653A2025580A006B6579625B
:1008B0006F6172645F70726F746F636F6C3A202542
:1008C000580A00686F73745F6B6579626F61726458
:1008D0005F6C65647328293A2025580A000A092D9F
:1008E00020537461747573202D0A004743433A20E6
:1008F000342E392E32204156522D4C4942433A2053
:10090000312E382E3073766E204156525F4152435D
:10091000483A2061767233350A004F5054494F4EA1
:10092000533A204C554641204D4F5553454B455960
:100930002045585452414B455920434F4E534F4C3C
:100940004520434F4D4D414E44204B45594D41505C
:100950005F53454354494F4E20343039360A0042E4
:1009600055494C443A20643030643765382D646909
:10097000727479202831303A31363A3334204A6162
:100980006E2031392032303138290A005649443A34
:100990002030784645454428742E6D2E6B2E292034
:1009A0005049443A20307830414442284144422062
:1009B0006B6579626F61726420636F6E76657274C5
:1009C000657229205645523A203078303130310A4C
:1009D00000444553433A20636F6E7665727420413C
:1009E0004442206B6579626F61726420746F205598
:1009F00053420A000A092D2056657273696F6E20F2
:100A00002D0A000A6D6F7573653A206F66660A00DD
:100A10000A6D6F7573653A206F6E0A000A6B65790F
:100A2000626F6172643A206F66660A000A6B6579CC
:100A3000626F6172643A206F6E0A000A6D617472AF
:100A400069783A206F66660A000A6D617472697887
:100A50003A206F6E0A000A64656275673A206F6E0D
:100A60000A000A64656275673A206F66660A000AC2
:100A70000A626F6F746C6F616465722E2E2E200097
:100A8000433E200011241FBECFEFD4E0DEBFCDBF18
:100A900004B603FE27C08091600290916102A0918C
:100AA0006202B09163028730904BA740B04BD1F403
:100AB0001092600210926102109262021092630220
:100AC00014BE84B7877F84BF0FB6F894A895809131
:100AD0006000886180936000109260000FBEE0E0CB
:100AE000F8E3099511E0A0E0B1E0E2EAFFE402C01A
:100AF00005900D92A433B107D9F722E0A4E3B1E049
:100B000001C01D92A036B207E1F70E94570C0C9469
:100B1000CF270C940000FF93EF93E0913401F09104
:100B20003501309709F00995EF91FF910895FC0187
:100B30008591803011F0EFDFFBCF0895FF27E0E2D1
:100B400030E247FF0CC0419597FF09C0EDE2609588
:100B5000709580959095611D711D811D911D27FFD8
:100B600002C0219530E350E2AA27660F771F881F45
:100B7000991FAA1FA41710F0A41B63955A95A9F7F3
:100B8000AA3008F0A95FA05DAF93F39561157105D8
:100B90008105910541F7ED3211F4EF93F395F217CA
:100BA00018F43F93F395FBCF8F91B5DFFA95E1F7FA
:100BB0000895E991F9918591803021F0853219F0FD
:100BC000AADFF9CF089520E0E89455915532C1F39A
:100BD000503311F4689455915A3348F4505390F3BC
:100BE000220F022E220F220F200D250FF4CF0EF41C
:100BF000219589919991533619F3533729F153353A
:100C000059F1BC0188279927E8945C3621F4899131
:100C1000999168945591543639F446EF7EF077FFF8
:100C20000DC08FEF9FEF0AC055374AE039F05835B5
:100C300040E121F0523642E009F00895FF93EF932E
:100C40007DDFEF91FF91B7CFFF93EF93FC0181918F
:100C50008030B9F360DFFBCFFF93EF9368DFF1CF14
:100C6000DF93CF93CDB7DEB72596A3DFCF91DF918A
:100C70000895282F2770E82FE695E695E695EF7002
:100C8000F0E0E05CFE4F87FF0AC081E090E001C029
:100C9000880F2A95EAF780959081892308C081E022
:100CA00090E001C0880F2A95EAF79081892B808314
:100CB00008950F931F93CF93DF93569A5E9A0E94E5
:100CC00050092FEF87EA91E6215080409040E1F7EC
:100CD00000C0000083E392E09F938F930E94300650
:100CE0000F900F90C1E0D0E009E112E063E08C2F9B
:100CF0000E945409009771F09F938F93DF93CF93D5
:100D00001F930F930E9430060F900F900F900F903B
:100D10000F900F909FEF29EF80E09150204080408E
:100D2000E1F700C000002196C031D105F9F663E07B
:100D300082E00E94540999278131910511F174F4E0
:100D400087309105F1F024F404970297F0F419C06C
:100D500089309105B1F00D97C1F413C08D31910523
:100D600081F034F48431910561F0499771F409C040
:100D7000843C910531F0873C910519F0813C910547
:100D800021F481E08093500102C01092500163E091
:100D900087E00E94540991E0823009F090E090933E
:100DA0005101992341F086E092E09F938F930E9436
:100DB00030060F900F9023E042E063E082E00E9453
:100DC000D40989EF91E09F938F930E9430060F9092
:100DD0000F90C1E0D0E00FED11E063E08C2F0E9496
:100DE0005409009771F09F938F93DF93CF931F93D4
:100DF0000F930E9430060F900F900F900F900F905E
:100E00000F908FEF99EF20E0815090402040E1F764
:100E100000C000002196C031D105F9F6E0E4F1E010
:100E200080E18E0F11928E13FDCF0E9454110E940B
:100E3000F708809142028160809342028FEC91E03A
:100E40000E949705569A5E98DF91CF911F910F915E
:100E50000895CF93DF938091390190913A010E94D8
:100E6000171F0C9708F4CCC00E94FF1E90933A0104
:100E7000809339010E94D009EC01009711F481E0C0
:100E8000BDC097FD05C080913B01816080933B010F
:100E9000D7FF05C080913B018E7F80933B01ED2FF2
:100EA000FF27EF73FF27CE018F739927C6FF02C07C
:100EB00080549109D6FF02C0E054F109A091380195
:100EC0000A2E000CBB0BBD010E94842781382FEF36
:100ED000920714F481E89FEF22273327281B390B50
:100EE00021388FEF380714F421E83FEF2195209344
:100EF0003C01CF01BD010E94842781382FEF92076A
:100F000014F481E89FEF91958195910981382FEF35
:100F1000920714F481E89FEF819580933D018091C1
:100F2000420283FF60C089EB91E00E949705DF9346
:100F3000CF9383EB91E09F938F930E94300681EBD8
:100F400091E00E94970580EA91E00E9497058091C8
:100F50003801282F082E000C330B3F938F938BE919
:100F600091E09F938F930E94300689E991E00E945F
:100F7000970580913B011F928F9384E991E09F93A5
:100F80008F930E94300682E991E00E94970580913C
:100F90003C01282F082E000C330B3F938F938FE8D2
:100FA00091E09F938F930E9430068DE891E00E941C
:100FB000970580913D01282F082E000C330B3F939D
:100FC0008F938AE891E09F938F930E94300687E881
:100FD00091E00E9497058DB79EB744960FB6F8949E
:100FE0009EBF0FBE8DBF8BE391E00E94A91180913F
:100FF000380191E088300CF090E0890F809338013F
:10100000DF91CF9108951F93CF93DF93C09100019B
:10101000D09101018FEF9FEF909301018093000128
:10102000CF3F8FEFD80709F074C0809136019091BF
:1010300037010E94171F0C9710F480E0CEC00E9469
:10104000FF1E909337018093360182E00E94CD0904
:10105000EC01892B09F05DC080915101882309F4CE
:1010600058C087E00E94CD09009709F452C09C0146
:101070002F77332722303105A1F048F421153105AF
:1010800069F02130310599F480788A641AC02330E0
:10109000310551F02F373105A1F009C08078826405
:1010A00010C0807889640DC0807888640AC084E7A5
:1010B00091E09F938F930E9430060F900F9081E1F3
:1010C0008CC0292F33272F7733272130310579F032
:1010D00050F02230310579F02330310581F4EC01F4
:1010E000D078D86416C0EC01D078D26412C0EC017C
:1010F000D078DA640EC0EC01D078D9640AC081E6F9
:1011000091E09F938F930E9430060F900F9080E1A3
:1011100064C08091420281FF18C0209709F48DCFEE
:101120008DE491E00E949705DF93CF9388E491E0EE
:101130009F938F930E94300686E491E00E9497056A
:101140000F900F900F900F9003C0209709F475CF68
:10115000CF378FE7D80711F48FE705C0CF3F8FEF68
:10116000D80721F48FEF0E94390636C02D2F332780
:10117000822F1C2F2F3F310581F4DF93CF9388E21C
:1011800091E09F938F930E9430060E9459060F9022
:101190000F900F900F908C2F20C0909150019923A9
:1011A00081F0A9014F7755274233510521F420786A
:1011B000822F8A6006C04A30510519F42078822FA8
:1011C00082630E9439061F3F39F0DC2FCC27CF6F96
:1011D000D0930101C093000181E0DF91CF911F9175
:1011E0000895E82FF0E0E05CFE4F80810895682FBD
:1011F000609582E00C940D0A509A83E091E001978B
:10120000F1F700C0000050989AEB9A95F1F700C0F2
:101210000895509A8AEB8A95F1F700C0509883E0C0
:1012200091E00197F1F700C000000895EF92FF925E
:101230000F931F93CF93DF93C0E0D0E090E8E92EA7
:10124000F12C082F10E0C7010C2E02C09595879550
:101250000A94E2F780239123892B19F00E9409094F
:1012600002C00E94FC082196C830D10561F7DF91C9
:10127000CF911F910F91FF90EF900895489B06C06A
:1012800023E02A95F1F700000197C1F708954899E6
:1012900006C023E02A95F1F700000197C1F70895F1
:1012A0005898509808950895CF92DF92EF92FF9248
:1012B0000F931F93CF93DF9300D0CDB7DEB7F89491
:1012C000509AE3EFFBE03197F1F700C000006A832A
:1012D00089830E9409096A816C6089818295807F77
:1012E000862B0E9416090E94FC0884EF91E00E9460
:1012F0004709892B21F4789482EE9FEF43C084EF55
:1013000091E00E943E09009711F478943BC011E1EE
:10131000C12CD12C02E882E890E00E9447097C01B0
:10132000882351F199270E943E09882329F1CC0C8A
:10133000DD1C902F9E19E81A9E1518F46894C0F8C9
:1013400006C0113121F478948CEE9FEF1BC0115030
:1013500011F78FE591E00E944709892B21F47894D9
:101360008BEE9FEF0FC08BE590E00E943E09892B2A
:10137000B1F77894C60106C07894812F90E09195DA
:10138000819591090F900F90DF91CF911F910F914F
:10139000FF90EF90DF90CF90089560E00C94540997
:1013A00060E083E00C9454091F93CF93DF9300D047
:1013B0001F92CDB7DEB7182FF894509A83EF9BE0B9
:1013C0000197F1F700C000002B834A8369830E94D4
:1013D00009096981862F88601295107F812B0E94F0
:1013E00016090E94FC088FE193E00197F1F700C015
:1013F00000000E9409094A81842F0E9416092B814E
:10140000822F0E9416090E94FC0878940F900F907A
:101410000F90DF91CF911F910895262F277040E004
:1014200062E00C94D40980915E0108959FB7F8940E
:10143000109255019FBF90915702943009F057C008
:101440009091E9009F703091EC00232F217030FDC6
:1014500020E8922B24E02093E9002091EB0020FF6C
:1014600043C02091EE0027FF3FC02091520122236C
:1014700021F02091E80025FF37C01092520126E0AC
:101480003091E80035FD15C030915702343061F5D8
:101490003091EB0035FD28C0215021F481E080938C
:1014A000520122C0EFE9FFE03197F1F700C00000E0
:1014B000E7CF8093F1008091E80085FD0AC080911C
:1014C000E80080FFFCCF8091E8008E778093E800F1
:1014D00006C08FB7F89421E0209355018FBF9F700D
:1014E0009093E90080E008959F709093E9008FEF5A
:1014F0000895CF93DF9300D01F92CDB7DEB79C0144
:1015000080915702843019F593E099833B832A83B5
:101510009093E9008FEF9091E800815095FD06C00F
:1015200095ED9A95F1F700008111F5CF8091E800D3
:1015300085FF0DC040E050E063E070E0CE01019611
:101540000E94190D8091E8008E778093E8000F903B
:101550000F900F90DF91CF910895CF93DF9300D03C
:101560001F92CDB7DEB720915702243021F522E03B
:1015700029839B838A8383E08093E9008FEF909196
:10158000E800815095FD06C095ED9A95F1F70000B1
:101590008111F5CF8091E80085FF0DC040E050E05B
:1015A00063E070E0CE0101960E94190D8091E80081
:1015B0008E778093E8000F900F900F90DF91CF917E
:1015C0000895209157022430F1F422E02093E9009D
:1015D0002FEF3091E800215035FD06C035ED3A95EA
:1015E000F1F700002111F5CF2091E80025FF0BC095
:1015F00040E050E065E070E00E94190D8091E80045
:101600008E778093E8000895CF93DF93209157025F
:10161000243039F521E02093E9002FEF3091E800E4
:10162000215035FD06C035ED3A95F1F70000211146
:10163000F5CF2091E80025FF14C0EC0140E050E018
:1016400068E070E00E94190D8091E8008E77809329
:10165000E80088E0FE01A6E5B1E001900D928A95D0
:10166000E1F7DF91CF9108950895209153012F5F05
:10167000822F62E30E949527992319F0209353014A
:1016800008951092530180915501882371F1809142
:101690005702843041F58091E9008F702091EC0071
:1016A000922F917020FD90E8892B94E09093E900AF
:1016B0009091EB0090FF14C09091EE0097FF10C046
:1016C0009091E80095FF03C01092F100F9CF90913E
:1016D000E80090FF05C09091E8009E779093E800A5
:1016E0008F708093E90010925501089542E061ECFB
:1016F00081E00E94220E42E061EC82E00E94220E14
:1017000042E061EC83E00E94220E42E261EC84E060
:101710000C94220E80915902833009F453C030F4A6
:10172000813071F0823009F48CC008958A3009F458
:1017300078C08B3009F45EC0893009F09AC020C0AF
:1017400080915802813A09F094C08091E800877F27
:101750008093E80080915C0290915D02892B21F4D6
:1017600068E086E591E003C060E080E090E070E032
:101770000E94640D8091E8008B778093E8000895C3
:1017800080915802813209F074C080915C0290917E
:101790005D02892B09F06DC08091E800877F8093FE
:1017A000E8008091E80082FD05C080915702811118
:1017B000F8CF5FC08091F10080935E018091E800D6
:1017C0008B7753C080915802813A09F052C08091C2
:1017D0005C0290915D02892B09F04BC08091E8007A
:1017E000877F8093E8008091E80080FFFCCF8091A4
:1017F0000C0136C0809158028132D9F580915C028B
:1018000090915D02892BA9F58091E800877F8093F4
:10181000E8000E94570E80915A0280930C010C94AC
:10182000ED1780915802813221F58091E800877F81
:101830008093E8000E94570E80915B0280935F01C5
:10184000089580915802813AA1F48091E800877F41
:101850008093E8008091E80080FFFCCF80915F01D9
:101860008093F1008091E8008E778093E8000C94DB
:10187000570E08950895089580915E018093540154
:1018800010925E0180E00E94F7080E94E7120C941B
:10189000ED170C943C0C0E948C1E809155028823FD
:1018A00029F00E94B51E81110C94030D089584B790
:1018B000877F84BF0FB6F894A895809160008861F7
:1018C00080936000109260000FBE90E080E80FB639
:1018D000F89480936100909361000FBE86E19AE0D6
:1018E0000E94611E83E692E00E9497050E943A0CD6
:1018F0000E9410120E94A80E0E94FB0E8091E2002E
:1019000084608093E2007894809157028430E1F7FC
:1019100082E592E00E9497050E94121282E091E017
:101920000E944F1181E492E00E9497050E943B0CB7
:1019300080915702853019F40E944B0CF9CF0E9418
:101940001812F6CF0E94C91E8091540180935E0147
:1019500008950C94A20C292F332723303105C9F0A8
:1019600064F42130310581F02230310509F043C0A3
:1019700084E790E02FEA32E042C021323105F1F0F5
:101980002232310541F137C082E190E023E233E0B9
:1019900036C099278130910541F08230910541F0A0
:1019A000892B49F5EBEAF2E005C0EBE9F2E002C071
:1019B000EBE6F2E0849190E09F0121C06430D8F41E
:1019C000E62FF0E0EE0FFF1FEF5DFE4F208131812B
:1019D00089E090E014C0643070F470E0FB01EE0F19
:1019E000FF1FE75EFE4F20813181FB01EB5EFE4F62
:1019F000808190E004C080E090E020E030E0FA01D7
:101A000031832083089584E089BD86E089BD09B4CF
:101A100000FEFDCF8091D8008F7D8093D80080910B
:101A2000E00082608093E0008091E00081FDFCCFC7
:101A30000895CF92DF92EF92FF920F931F93CF936F
:101A4000DF93EC018B016A010E94760E811133C095
:101A5000C114D10439F0F60180819181081B190B62
:101A6000C80FD91FE12CF12C0115110519F1809136
:101A7000E80085FD16C08091E8008E778093E8002D
:101A8000C114D10449F0F60180819181E80EF91E5C
:101A9000F182E08285E00FC00E94760E882321F358
:101AA0000AC089918093F10001501109FFEFEF1AEC
:101AB000FF0ADACF80E0DF91CF911F910F91FF9065
:101AC000EF90DF90CF90089520915E0230915F02F9
:101AD0002617370748F06115710539F42091E800A1
:101AE0002E772093E80001C0B90140E0611571052F
:101AF00091F120915702222309F440C0253009F4C6
:101B00003FC02091E80023FD3DC02091E80022FD68
:101B10002FC02091E80020FFE9CF2091F20030E0B3
:101B2000FC01CF016115710559F02830310540F4F1
:101B300081918093F100615071092F5F3F4FF1CF88
:101B400041E02830310509F040E02091E8002E778F
:101B50002093E800CBCF4111CCCF0AC0809157022F
:101B6000882361F0853061F08091E80083FD0AC030
:101B70008091E80082FFF2CF80E0089582E008952E
:101B800083E0089581E0089520915E0230915F0224
:101B90002617370748F06115710539F42091E800E0
:101BA0002E772093E80001C0B901FC0120E0611507
:101BB000710579F180915702882309F43DC0853081
:101BC00009F43CC08091E80083FD3AC08091E800B0
:101BD00082FD2CC08091E80080FFE9CF8091F20067
:101BE00090E06115710559F08830910540F4249119
:101BF0002093F1003196615071090196F2CF21E0F6
:101C0000089709F020E08091E8008E778093E80043
:101C1000CECF2111CFCF0AC080915702882361F027
:101C2000853061F08091E80083FD0AC08091E80072
:101C300082FFF2CF80E0089582E0089583E0089566
:101C400081E00895982F953058F59093E900981702
:101C500039F07091EC002091ED005091F00003C03C
:101C6000242F762F50E021FF19C03091EB003E7FEA
:101C70003093EB003091ED003D7F3093ED003091DB
:101C8000EB0031603093EB007093EC002093ED009B
:101C90005093F0002091EE0027FF07C09F5FD3CF45
:101CA0008F708093E90081E0089580E0089580912D
:101CB000580287FF11C08091E80082FD05C0809125
:101CC00057028111F8CF11C08091E8008B770BC0CB
:101CD00080915702882349F08091E80080FFF8CF77
:101CE0008091E8008E778093E80008952091E400C9
:101CF0003091E50095E64091EC00842F817040FF23
:101D000022C08091E80080FD1CC08091570288238A
:101D100091F0853091F08091EB0085FD10C04091ED
:101D2000E4005091E5004217530729F39A019150BE
:101D300011F784E0089582E0089583E0089581E03A
:101D4000089580E008954091E80042FFDECF0895B5
:101D50000E94050F0E94080FE0EEF0E08081816094
:101D60008083E8EDF0E080818F77808319BCE3E623
:101D7000F0E08081816080831092560208950E9475
:101D8000050F0E94080F8091D8008F778093D800AC
:101D90008091D80080688093D8008091D8008F7D92
:101DA0008093D80084E089BD86E089BD09B400FE37
:101DB000FDCF1092570210925302109255021092CA
:101DC000540242E060E080E00E94220E8091E10037
:101DD0008E7F8093E1008091E20081608093E20039
:101DE0008091E20088608093E2008091E0008E7F25
:101DF0008093E0000895E3E6F0E080818E7F8083A9
:101E000081E0809356020C94BF0E1092E200089578
:101E10001092E10008951F920F920FB60F921124B5
:101E20002F933F934F935F936F937F938F939F93E2
:101E3000AF93BF93EF93FF938091E10082FF0BC0BC
:101E40008091E20082FF07C08091E1008B7F809348
:101E5000E1000E94350B8091E10080FF19C0809164
:101E6000E20080FF15C08091E2008E7F8093E20047
:101E70008091E20080618093E2008091D8008062CE
:101E80008093D80019BC85E0809357020E94490CCA
:101E90008091E10084FF30C08091E20084FF2CC07B
:101EA00084E089BD86E089BD09B400FEFDCF809144
:101EB000D8008F7D8093D8008091E1008F7E809341
:101EC000E1008091E2008F7E8093E2008091E20049
:101ED00081608093E20080915302882311F084E0B6
:101EE00007C08091E30087FD02C081E001C083E06C
:101EF000809357020E94A90C8091E10083FF29C0C2
:101F00008091E20083FF25C08091E100877F80936C
:101F1000E10082E080935702109253028091E10029
:101F20008E7F8093E1008091E2008E7F8093E200BB
:101F30008091E20080618093E20042E060E080E016
:101F40000E94220E8091F00088608093F0000E9431
:101F5000340BFF91EF91BF91AF919F918F917F9142
:101F60006F915F914F913F912F910F900FBE0F9006
:101F70001F9018951F920F920FB60F9211242F9356
:101F80003F934F935F936F937F938F939F93AF9301
:101F9000BF93CF93DF93EF93FF93C091E900CF708E
:101FA0008091EC00D82FD17080FDD0E81092E9002C
:101FB0008091F000877F8093F00078940E94FE0F5C
:101FC0001092E9008091F00088608093F000CD2BA2
:101FD000CF70C093E900FF91EF91DF91CF91BF9156
:101FE000AF919F918F917F916F915F914F913F91B1
:101FF0002F910F900FBE0F901F9018951F93CF93A6
:10200000DF93CDB7DEB7AA970FB6F894DEBF0FBE49
:10201000CDBFE8E5F2E088E08E0F9091F10091935A
:102020008E13FBCF0E948A0B8091E80083FF1FC1B3
:102030008091580290915902492F50E04A30510541
:1020400008F015C1FA01E65CFF4F0C94B527803803
:1020500081F0823809F00BC180915C028F7080930F
:10206000E9008091EB0085FB882780F91092E90058
:1020700006C0809154029091550291118260909116
:10208000E800977F9093E8008093F1001092F100B0
:10209000C8C0282F2D7F09F0EAC0882319F08230AC
:1020A00061F0E5C080915A02813009F0E0C09330C0
:1020B00009F080E0809355022BC080915A02811173
:1020C00027C080915C028F7009F4D1C08093E90031
:1020D0002091EB0020FF1CC0933021F48091EB0095
:1020E000806214C09091EB0090619093EB0021E02E
:1020F00030E0A90102C0440F551F8A95E2F74093D2
:10210000EA001092EA008091EB0088608093EB0077
:102110001092E9008091E800877F86C08111A7C0F6
:1021200010915A021F778091E3008078812B809371
:10213000E3008091E800877F8093E8000E94570EBB
:102140008091E80080FFFCCF8091E300806880935D
:10215000E300111102C082E001C083E080935702C6
:1021600086C08058823008F082C080915A029091D7
:102170005B028C3D53E0950779F583E08A838AE220
:1021800089834FB7F894DE01139620E03EE051E2D8
:10219000E32FF0E050935700E49120FF03C0E29555
:1021A000EF703F5FEF708E2F90E0EA3010F0C7962F
:1021B00001C0C0968D939D932F5F243149F74FBF87
:1021C0008091E800877F8093E8006AE270E0CE01AA
:1021D00001960E94640D14C0AE014F5F5F4F609185
:1021E0005C020E94AB0CBC01892B09F440C09091A9
:1021F000E800977F9093E80089819A810E94C40D3E
:102200008091E8008B778093E80031C0803879F5C1
:102210008091E800877F8093E8008091530280934B
:10222000F1008091E8008E778093E8000E94570EBD
:102230001EC081111CC090915A029230C0F480914E
:10224000E800877F8093E800909353020E94570E26
:1022500080915302811106C08091E30087FD02C086
:1022600081E001C084E0809357020E94760B809148
:10227000E80083FF0AC08091E800877F8093E80030
:102280008091EB0080628093EB00AA960FB6F894E1
:10229000DEBF0FBECDBFDF91CF911F910895909308
:1022A0006501809364010895E0916401F0916501F6
:1022B000309721F00190F081E02D099480E008959D
:1022C000EF92FF920F931F93CF93DF93E0916401FE
:1022D000F09165013097B1F18C010280F381E02D1E
:1022E00009958091420282FF2DC080FF04C080E4E6
:1022F00094E00E949705E80118E08AE3E82E84E064
:10230000F82E8091420280FF0BC088811F928F932C
:10231000FF92EF920E9430060F900F900F900F9057
:10232000115021961111EDCF8091420280FF0AC019
:1023300088E394E0DF91CF911F910F91FF90EF9090
:102340000C949705DF91CF911F910F91FF90EF9023
:102350000895E0916401F0916501309721F00480C7
:10236000F581E02D09940895CF93DF93EC018091DE
:10237000620190916301C817D90709F1D0936301F5
:10238000C0936201E0916401F09165013097B9F06A
:102390000680F781E02DCE0109958091420282FFEF
:1023A0000EC080FF0CC0DF93CF938AE294E09F932E
:1023B0008F930E9430060F900F900F900F90DF9137
:1023C000CF910895CF93DF93EC01809160019091BC
:1023D0006101C817D90709F1D0936101C093600169
:1023E000E0916401F09165013097B9F00084F185C6
:1023F000E02DCE0109958091420282FF0EC080FF40
:102400000CC0DF93CF938AE194E09F938F930E9457
:1024100030060F900F900F900F90DF91CF9108959D
:102420000C94E8120E94F61E0E9459060C9453095F
:102430005F926F927F928F929F92AF92BF92CF9254
:10244000DF92EF92FF920F931F93CF93DF9300D011
:1024500000D01F92CDB7DEB70E94030887E6C82ED2
:1024600081E0D82E512C88248394912C852D0E94B4
:10247000F108A82EF601E080E82641F45394FFEF1E
:10248000CF1ADF0A80E15812F1CF40C0809142029A
:1024900081FD0E94041300E010E0F12CB12CC70173
:1024A000002E02C0959587950A94E2F780FF28C018
:1024B00009835A823401002E02C0660C771C0A94EC
:1024C000E2F793012A213B2181E0232B09F480E0EC
:1024D0008B830E94FF1E8160782F9D838C834981AE
:1024E0005A816B818D810E943A1349815A816B8197
:1024F0007C818D810E94791EF60180816826608230
:102500000F5F1F4F0830110551F6B8CF8FEF898349
:102510008A831B820E94FF1E8160782F9D838C839B
:1025200049815A816B818D810E943A130E94781EE5
:102530000E94CC210E942907109166010E9454112B
:10254000181771F10E945411809366019091420214
:1025500092FF0EC090FF0CC01F928F938BE494E00B
:102560009F938F930E9430060F900F900F900F90C3
:10257000809166010F900F900F900F900F90DF9158
:10258000CF911F910F91FF90EF90DF90CF90BF9070
:10259000AF909F908F907F906F905F900C948A1E69
:1025A0000F900F900F900F900F90DF91CF911F9190
:1025B0000F91FF90EF90DF90CF90BF90AF909F90E2
:1025C0008F907F906F905F9008950C94F708089516
:1025D0000895CF93DF931F92CDB7DEB769830E9432
:1025E000F10890E021E030E0698102C0220F331F42
:1025F0006A95E2F72823392381E0232B09F480E050
:102600000F90DF91CF910895EF92FF920F931F9358
:10261000CF93DF9384E694E00E949705C0E0D0E07A
:1026200089E2E82E81E0F82E06E514E08C2F0E9466
:10263000F1080E94661EFF92EF921F928F93DF9324
:10264000CF931F930F930E94300621968DB79EB7AC
:1026500008960FB6F8949EBF0FBE8DBFC031D1054E
:1026600029F7DF91CF911F910F91FF90EF9008957F
:1026700008950895CF93DF93CDB7DEB72B970FB6AC
:10268000F894DEBF0FBECDBF942F4F83252F588700
:1026900069877A878B874A855B85452B21F02F3F99
:1026A00009F59F3FF9F4DE01119686E0FD011192D4
:1026B0008A95E9F785E0FE01379601900D928A959B
:1026C000E1F749815A816B817C818D819E810E94D5
:1026D000DF1A2B960FB6F894DEBF0FBECDBFDF9189
:1026E000CF9108954F81588569857A858B850E94A1
:1026F000791ED9CFCF93882309F4A9C0C82F823877
:10270000A1F40E94541181FDA2C089E30E94C21D60
:102710000E943B1E2FEF81EE94E0215080409040BC
:10272000E1F700C0000089E315C08338C1F40E94BE
:10273000541180FD8CC083E50E94C21D0E943B1E87
:102740002FEF81EE94E0215080409040E1F700C0EF
:10275000000083E50E94DF1DCF910C943B1E84385E
:10276000A1F40E94541182FD72C087E40E94C21D30
:102770000E943B1E2FEF81EE94E02150804090405C
:10278000E1F700C0000087E4E5CF8CEF8C0F813AC1
:1027900020F080E58C0F8E3248F48C2F0E94F824B4
:1027A000811155C08C2F0E94C21DD6CF80E28C0FA4
:1027B000883048F4C77081E001C0880FCA95EAF7F5
:1027C0000E94011EC9CF8BE58C0F833078F4C53A87
:1027D00029F0C63A31F083E890E005C081E890E046
:1027E00002C082E890E0CF910C94B41188E58C0F80
:1027F000853168F5C83A89F0C93A91F0CA3A99F03A
:10280000CB3AA1F0CC3AA9F0CD3AB1F0CE3AB9F03A
:10281000CF3AC1F080E090E017C082EE90E014C0A3
:1028200089EE90E011C08AEE90E00EC085EB90E05A
:102830000BC086EB90E008C083EB90E005C084EB12
:1028400090E002C087EB90E0CF910C94E211CF9121
:102850000895882309F46AC08238A1F40E945411B3
:1028600081FF64C089E30E94C21D0E943B1E2FEFBE
:1028700081EE94E0215080409040E1F700C00000DC
:1028800089E315C08338B9F40E94541180FF4EC00B
:1028900083E50E94C21D0E943B1E2FEF81EE94E053
:1028A000215080409040E1F700C0000083E50E9485
:1028B000DF1D0C943B1E8438A1F40E94541182FF4A
:1028C00035C087E40E94C21D0E943B1E2FEF81EE9F
:1028D00094E0215080409040E1F700C0000087E480
:1028E000E6CF9CEF980F913A10F390E5980F9E3247
:1028F000F0F290E2980F983050F4877091E001C0A8
:10290000990F8A95EAF7892F0E94071ED2CF9BE57F
:10291000980F933020F480E090E00C94B411885A22
:10292000853120F480E090E00C94E2110895882332
:1029300021F00E94011E0C943B1E0895882321F073
:102940000E94071E0C943B1E0895BF92CF92DF9207
:10295000EF92FF920F931F93CF93DF9300D000D09D
:1029600000D0CDB7DEB725E0FC01DE011196019065
:102970000D922A95E1F7FC0140815181028163812A
:102980007481258122952F706115710509F403C3A7
:102990005F3F19F44F3F09F4FEC26C01862F7D831F
:1029A0006C83602F782F8D812E830E943F1D182FFE
:1029B000B92E0E943E1D0E942E1CEB2DE295EF7059
:1029C000F0E0EC5BFF4F2E810C94B5278B2D807FC0
:1029D0009B2D9F70F92E882319F0F29490EFF92225
:1029E000002349F0FF2009F483C28F2D0E94141E9A
:1029F0000E943B1E7DC2812F0E942914FF2009F4F2
:102A0000CAC28F2D0E941A1E26960FB6F894DEBFFA
:102A10000FBECDBFDF91CF911F910F91FF90EF902F
:102A2000DF90CF90BF900C943B1E8B2D807F9B2D11
:102A30009F70F92E803219F0F29480EFF822112362
:102A400019F0113009F12AC00023B1F08F2D222393
:102A500051F1213041F526960FB6F894DEBF0FBE36
:102A6000CDBFDF91CF911F910F91FF90EF90DF903D
:102A7000CF90BF900C94241E222319F0213009F42A
:102A80008AC20E94271E2DC00023F1F0263008F0D4
:102A900082C20E94FE1D8F2129F023C00023F9F07D
:102AA000211116C08F2D26960FB6F894DEBF0FBEEB
:102AB000CDBFDF91CF911F910F91FF90EF90DF90ED
:102AC000CF90BF900C949714253008F064C209C0D1
:102AD000F601858180FF0CC28F708583E3CF2111C1
:102AE0001CC28F2D83C12B2D26952695237030E097
:102AF0002115310521F021303105D1F04CC20023E0
:102B000021F0812F9B2D937002C080E090E02696EB
:102B10000FB6F894DEBF0FBECDBFDF91CF911F91EE
:102B20000F91FF90EF90DF90CF90BF900C94B41175
:102B3000002321F0812F9B2D937002C080E090E054
:102B400026960FB6F894DEBF0FBECDBFDF91CF91B2
:102B50001F910F91FF90EF90DF90CF90BF900C945A
:102B6000E211812F002319F00E94522002C00E941E
:102B7000BA2026960FB6F894DEBF0FBECDBFDF9108
:102B8000CF911F910F91FF90EF90DF90CF90BF906A
:102B90000C943F218B2D837009F07BC00111FBC188
:102BA000812F829586958770880F880F912F9F704F
:102BB000C92ED12CE12CF12C082E04C0CC0CDD1C2C
:102BC000EE1CFF1C0A94D2F714FF12C04FE050E035
:102BD00060E070E004C0440F551F661F771F8A95A0
:102BE000D2F7CB01BA01609570958095909503C09E
:102BF00060E070E0CB012B2D269526952370422FA7
:102C000050E042305105D9F04330510569F16C294B
:102C10007D298E299F294130510551F126960FB605
:102C2000F894DEBF0FBECDBFDF91CF911F910F9102
:102C3000FF90EF90DF90CF90BF900C94531C6C29C5
:102C40007D298E299F2926960FB6F894DEBF0FBEE8
:102C5000CDBFDF91CF911F910F91FF90EF90DF904B
:102C6000CF90BF900C946D1C0E94531CC701B601FD
:102C700026960FB6F894DEBF0FBECDBFDF91CF9181
:102C80001F910F91FF90EF90DF90CF90BF900C9429
:102C9000391C002319F08B2D817001C08695882383
:102CA00009F479C1812F829586958770880F880FE6
:102CB000912F9F70C92ED12CE12CF12C082E04C02D
:102CC000CC0CDD1CEE1CFF1C0A94D2F714FF12C0C2
:102CD0004FE050E060E070E004C0440F551F661FF5
:102CE000771F8A95D2F7CB01BA01609570958095D0
:102CF000909503C060E070E0CB012B2D26952695C2
:102D00002370422F50E042305105D9F04330510535
:102D100069F16C297D298E299F294130510551F196
:102D200026960FB6F894DEBF0FBECDBFDF91CF91D0
:102D30001F910F91FF90EF90DF90CF90BF900C9478
:102D40001A1D6C297D298E299F2926960FB6F89485
:102D5000DEBF0FBECDBFDF91CF911F910F91FF90CE
:102D6000EF90DF90CF90BF900C942C1D0E941A1D05
:102D7000C701B60126960FB6F894DEBF0FBECDBFD1
:102D8000DF91CF911F910F91FF90EF90DF90CF9047
:102D9000BF900C94081D103FD1F128F480E4810FFE
:102DA000803250F0A0C0123F09F462C008F44BC05A
:102DB000133F09F472C097C0F12FF071FF2E8B2DD5
:102DC0008F71002351F00E94A11C812FFF2019F068
:102DD0008295807F68CE8F7066CE0E94C21C812F44
:102DE000FF2019F08295807F01C08F7026960FB664
:102DF000F894DEBF0FBECDBFDF91CF911F910F9131
:102E0000FF90EF90DF90CF90BF900C949E14002322
:102E1000B1F0253008F0BFC08B2D8F7126960FB60C
:102E2000F894DEBF0FBECDBFDF91CF911F910F9100
:102E3000FF90EF90DF90CF90BF900C94E71C26306E
:102E400008F0A9C0E9CF0023A9F08B2D8F71269639
:102E50000FB6F894DEBF0FBECDBFDF91CF911F91AB
:102E60000F91FF90EF90DF90CF90BF900C94A11C3A
:102E7000002359F38B2D8F7126960FB6F894DEBF81
:102E80000FBECDBFDF91CF911F910F91FF90EF90BB
:102E9000DF90CF90BF900C94C21C002399F08B2D33
:102EA0008F7126960FB6F894DEBF0FBECDBFDF91AF
:102EB000CF911F910F91FF90EF90DF90CF90BF9037
:102EC0000C948C1C26960FB6F894DEBF0FBECDBFB7
:102ED000DF91CF911F910F91FF90EF90DF90CF90F6
:102EE000BF900C94871C0023A9F0222309F4ADCFD6
:102EF000812F26960FB6F894DEBF0FBECDBFDF91AF
:102F0000CF911F910F91FF90EF90DF90CF90BF90E6
:102F10000C947A13222309F4ADCF812F26960FB695
:102F2000F894DEBF0FBECDBFDF91CF911F910F91FF
:102F3000FF90EF90DF90CF90BF900C9429144B2D11
:102F40004F70612FC6010E94C81F26960FB6F894D5
:102F5000DEBF0FBECDBFDF91CF911F910F91FF90CC
:102F6000EF90DF90CF90BF900C94871B4B2D4F704C
:102F7000612FC60126960FB6F894DEBF0FBECDBFF7
:102F8000DF91CF911F910F91FF90EF90DF90CF9045
:102F9000BF900C94CB1F26960FB6F894DEBF0FBEE1
:102FA000CDBFDF91CF911F910F91FF90EF90DF90F8
:102FB000CF90BF9008950E94211E0E94F01D0E9494
:102FC0003B1E0E9473220E943F2180E090E00E94FD
:102FD000B41180E090E00C94E2110E94111E0C9458
:102FE000DB17CF93DF9300D000D01F92CDB7DEB7B1
:102FF000942F4983252F5A836B837C838D834C8147
:103000005D81452B39F12F3F11F49F3F19F1498123
:103010005A816B817C818D810E943F1D292F2295D1
:103020002F7030E02C30310504F52A3031055CF486
:10303000225031092230310568F4853A80F4843019
:1030400090F4823080F0883E38F4803E60F4845002
:10305000813A48F080E014C0803FE1F704C090E27C
:10306000980F983080F781E00BC02C30310521F4A7
:1030700093FB882780F904C02F303105C9F3EACFCC
:103080000F900F900F900F900F90DF91CF910895B8
:10309000CF93DF9300D000D01F92CDB7DEB70F9053
:1030A0000F900F900F900F90DF91CF910895CF93D5
:1030B000DF9300D000D000D0CDB7DEB726960FB694
:1030C000F894DEBF0FBECDBFDF91CF910895CF93AF
:1030D000DF93C091770180917801C817A1F0D0E00B
:1030E000CE0166E070E00E948427FC01E758FE4FA5
:1030F0004081518162817381848195810E9457183A
:103100002196C770E8CFDF91CF9108954091A90132
:103110005091AA016091AB017091AC018091AD0119
:103120009091AE010C945718CF93DF938091AE012C
:1031300082958F7009F05CC08091AB01882309F4FF
:1031400057C020917701D09178014091A901C09199
:10315000AA01E091AC01F091AD012D1709F448C02E
:1031600030E0309709F440C0CF3F11F44F3FE1F118
:10317000C90166E070E00E948427DC01A758BE4FB9
:1031800011968C911197C8132FC08C9148132CC0A5
:1031900012968C911297811127C013968D919C9154
:1031A00014978E179F0708F401978E1B9F0B883C7E
:1031B0009105D0F48091AE018F7080618093AE0153
:1031C000C90166E070E00E948427FC01E258FE4FCE
:1031D00090819F709061908389EA91E00E94A5148C
:1031E000DF91CF910C9467182F5F3F4F2770B5CFB9
:1031F000DF91CF910895BF92CF92DF92EF92FF922D
:103200000F931F93CF93DF93CDB7DEB761970FB6C0
:10321000F894DEBF0FBECDBF7C0185E0F701DE0173
:103220001D9601900D928A95E1F7D7014C91119668
:103230002C9111971296DC90129713960D911C9178
:1032400014975091A9016091AA018091AC019091CD
:10325000AD01009709F481C16F3F19F45F3F09F494
:103260007CC1B090AB01BB2009F4CCC03091AE0161
:103270000817190728F0F801E81BF90BCF0104C063
:1032800080959095800F911FCC24C394883C910524
:1032900088F0C12C307F09F0D4C0702F198B088BB7
:1032A000522F6D2D89890E94481889EA91E00E9469
:1032B000A514BDC0832F807F09F04AC0621314C0DB
:1032C000541312C0D11010C03F7030613093AE0162
:1032D0000E94861889EA91E00E94A5148091AE01AF
:1032E000D70115968C9332C00115110531F12F3F8E
:1032F00011F44F3F11F1CD2CD1101FC0E091770197
:1033000030917801E31709F462C0F0E0CF0166E084
:1033100070E00E948427DC01A758BE4F11968C9163
:103320001197281307C08C91481304C012968C91F2
:10333000811103C03196E770E5CFCD2CDD2009F473
:103340002DC18091AE0181608093AE01C12C26C158
:10335000621308C0541306C0D11004C08091AE019E
:10336000D701CEC04D872E87DF86702F198B088B33
:10337000522F6D2D89890E94F117882309F43EC0D0
:10338000DD20E1F12091AE01822F82958F7090E0D7
:10339000029774F08091A9019091AA0198878F8378
:1033A00019861B870A872C87CE0107960E94A514D1
:1033B00086E0F701A9EAB1E001900D928A95E1F764
:1033C0000E9494180E948618CC24C394E7C0702FE2
:1033D000198B088B522F60E089890E943F1D292F8D
:1033E00022952F7030E0223031050CF0CBC09F7059
:1033F00009F0C5C0805E883008F4D0C0C7010E94C3
:10340000A514E2CF0817190708F458C0F801E81B03
:10341000F90BCF01883C910508F455C0C12C702FE1
:10342000198B088B522F6D2D89890E944818E9EA63
:10343000F1E086E0DF011D928A95E9F70E94861887
:10344000ADC0621314C0541312C0D11010C08091CB
:10345000AE01F7018583C7010E94A51486E0E9EA61
:10346000F1E0DF011D928A95E9F7CB2C97C04D87DB
:103470002E87DF86702F198B088B522F6D2D89892F
:103480000E94F117882309F4B9CFDD2009F4B6CFE3
:103490002091AE01822F82958F7090E002970CF4FC
:1034A00087CF8091A9019091AA019A8389831B8279
:1034B0001D830C832E83CE01019678CF8095909545
:1034C000800F911FA7CFCD2CDD2009F497CF621379
:1034D0002EC054132CC02091AE0120FD1FC0822F9E
:1034E00082958F70D9F0D70115962C9315978F3050
:1034F00049F08F5F982F9295907F822F8F70892B44
:1035000015968C93C7010E94A51486E0F701A9EADD
:10351000B1E001900D928A95E1F790CF86E0F70136
:10352000A9EAB1E001900D928A95E1F737C04D8785
:103530002E87DF86702F198B088B522F6D2D89896E
:103540000E94F117811134CF8091AE018160809388
:10355000AE01C7010E94A51421C0DD2009F44ECFA1
:103560004D872E87DF86702F198B088B522F6D2D7C
:1035700089890E94F117882309F440CF19CF81115E
:1035800039CF0CC0243031050CF038CF9F7009F4CE
:1035900031CFF7019581907F09F02CCF8C2D61966A
:1035A0000FB6F894DEBF0FBECDBFDF91CF911F9154
:1035B0000F91FF90EF90DF90CF90BF900895CF9341
:1035C000DF93CDB7DEB72C970FB6F894DEBF0FBEF2
:1035D000CDBF4F83588769877A878B879C87CE01B9
:1035E00007960E94FB18882371F08F8198852A85A1
:1035F0003B85232B09F43FC09F3F09F068C08F3FF4
:1036000009F065C038C086E0FE013796DE011196EC
:1036100001900D928A95E1F76F817885EA85FB85A7
:10362000309749F17F3F11F46F3F29F18091780184
:1036300090E09C012F5F3F4F277033274091770127
:1036400050E02417350709F44BC069837A83FD8362
:10365000EC8366E070E00E948427DC01A758BE4F2F
:1036600096E0FE01319601900D929A95E1F7209334
:1036700078010E94671880917701909178018917ED
:10368000E9F190E066E070E00E94842787589E4F41
:103690000E94FB18882391F18091770190E066E009
:1036A00070E00E948427FC01E758FE4F4081518161
:1036B00062817381848195810E945718809177017E
:1036C00090E001968770992780937701D4CF4F813E
:1036D000588569857A858B859C850E945718CBCF44
:1036E0000E94ED171092780110927701E9EAF1E05B
:1036F00086E0DF011D928A95E9F7BDCF2C960FB6C3
:10370000F894DEBF0FBECDBFDF91CF910895DF9259
:10371000EF92FF920F931F93CF93DF93FC01892BBE
:1037200009F48AC0E12CF12CDD24D394EF01219619
:103730008491853709F461C058F4843708F04EC08D
:10374000843008F06AC08130D1F0823071F174C0E9
:10375000883709F45DC050F4863709F455C08737BF
:1037600009F06AC08E2D0E940E1E54C09CE7980F6F
:10377000903708F061C08F770E94291450C08F01E4
:103780000E5F1F4FFE01849190E2980F983050F425
:103790008770FD2D01C0FF0F8A95EAF78F2F0E94D9
:1037A000141E14C00E947A1313C08F010E5F1F4FA6
:1037B000FE01C49180E28C0F883060F4C7708D2DBB
:1037C00001C0880FCA95EAF70E941A1E0E943B1E8C
:1037D000E80125C08C2F0E942914FACF9F012E5F8B
:1037E0003F4FFE01C491CC2369F08FE99FE0019720
:1037F000F1F700C00000C150F6CF9F012E5F3F4F90
:10380000FE01F490E9010BC00E94FE1DE82E07C0E6
:103810000E94111E0E943B1E02C00E947A138F2D2F
:10382000882341F0EFE9FFE03197F1F700C0000095
:103830008150F6CFFE017ACFDF91CF911F910F918A
:10384000FF90EF90DF90089560932F027093300205
:1038500080933102909332020C94891E08956093F4
:1038600033027093340280933502909336020C94A5
:10387000881E0F931F930091330210913402209100
:10388000350230913602602B712B822B932B609383
:1038900033027093340280933502909336021F9165
:1038A0000F910C94881E0F931F9300913302109177
:1038B0003402209135023091360260237123822335
:1038C0009323609333027093340280933502909374
:1038D00036021F910F910C94881E0F931F93009135
:1038E0003302109134022091350230913602602764
:1038F0007127822793276093330270933402809359
:103900003502909336021F910F910C94881E60E04F
:1039100070E0CB010C94241C0F931F9341E050E006
:1039200060E070E08A019B0104C0000F111F221F9C
:10393000331F8A95D2F7C901B8011F910F910C94DA
:10394000241C0F931F9341E050E060E070E004C03E
:10395000440F551F661F771F8A95D2F780912F025B
:1039600090913002A0913102B09132028A019B0104
:10397000082B192B2A2B3B2BC901B8011F910F9142
:103980000C94241C0F931F9341E050E060E070E022
:1039900004C0440F551F661F771F8A95D2F74095C4
:1039A00050956095709580912F0290913002A09172
:1039B0003102B09132028A019B01082319232A2384
:1039C0003B23C901B8011F910F910C94241C0F9344
:1039D0001F9341E050E060E070E004C0440F551FC9
:1039E000661F771F8A95D2F780912F02909130023F
:1039F000A0913102B09132028A019B010827192758
:103A00002A273B27C901B8011F910F910C94241C50
:103A10000F931F9300912F021091300220913102D9
:103A200030913202602B712B822B932B1F910F91BF
:103A30000C94241C0F931F9300912F0210913002BD
:103A4000209131023091320260237123822393232B
:103A50001F910F910C94241C0F931F9300912F0220
:103A6000109130022091310230913202602771278B
:103A7000822793271F910F910C94241C08958F92F5
:103A80009F92AF92BF92DF92EF92FF920F931F939C
:103A9000CF93DF9300D000D01F92CDB7DEB76B83FA
:103AA0007C838D838A018C819D81892B21F01F3F2E
:103AB00029F44F3F19F480E090E053C08B818823B4
:103AC00009F43CC08090330290903402A0903502FB
:103AD000B090360280912F0290913002A091310275
:103AE000B0913202882A992AAA2ABB2A2FE1E22E13
:103AF000F12CD501C4010E2C04C0B695A79597955D
:103B000087950A94D2F780FF07C0DE2CB8018E2D6E
:103B10000E94991F019729F481E0E81AF10848F7FB
:103B2000D12CE12FF0E093E0EE0FFF1F9A95E1F723
:103B3000E00FF11DE155FE4FD0820CC0E12FF0E007
:103B400083E0EE0FFF1F8A95E1F7E00FF11DE155CD
:103B5000FE4FD08009831A8369817A818D2D0E945E
:103B6000991F0F900F900F900F900F90DF91CF91B2
:103B70001F910F91FF90EF90DF90BF90AF909F90BB
:103B80008F90089520910D0130910E01F901329628
:103B90009FEF40E05191581789F09F3F19F4511160
:103BA00001C0942F4F5F4630A9F79F3F39F0F901CC
:103BB000E90FF11D97FDFA958283089508952091EC
:103BC0000D0130910E01F9013296285F3F4F90812F
:103BD000981301C010823196E217F307C1F70895D8
:103BE00081E090E0E0910D01F0910E01E80FF91FE6
:103BF0001082019688309105A9F7089580914102BD
:103C0000089590914102892B8093410208958095F7
:103C1000909141028923809341020895809341024B
:103C2000089510924102089590914002892B80934B
:103C3000400208958095909140028923809340022C
:103C400008951092400208958093370208951092CB
:103C50003702089580910D0190910E01FC0131967B
:103C60009C01285F3F4F80E0919191118F5FE21797
:103C7000F307D1F70895E0910D01F0910E018091C5
:103C800041028083E0910D01F0910E0190818091BD
:103C90004002892B808380913702882361F0E09174
:103CA0000D01F0910E019081892B80830E942A1EC4
:103CB00081111092370280910D0190910E010C94A8
:103CC0006011909335018093340108958295982F67
:103CD0009C7C292F26952695982F9373990F990FE1
:103CE000922B892F8A7A86959575990F892B08953D
:103CF0000895CF93DF9300D000D01F92CDB7DEB7E9
:103D00000F900F900F900F900F90DF91CF9108952B
:103D1000089508950C94E51280915702843021F1A2
:103D20001092430220E488E190E00FB6F894A89541
:103D3000809360000FBE2093600083B7817F846012
:103D400083BF83B7816083BF7894889583B78E7F64
:103D500083BF0FB6F894A895809160008861809326
:103D60006000109260000FBE0895CF930E94381338
:103D70000E9403080E943913C0E08C2F0E94F108B2
:103D8000811104C0CF5FC031C1F701C081E0CF9184
:103D900008950E94E7120C94ED171F920F920FB630
:103DA0000F9211248F939F93AF93BF9380914302FF
:103DB000811113C08091440290914502A091460266
:103DC000B09147024196A11DB11D8093440290938A
:103DD0004502A0934602B0934702BF91AF919F91D5
:103DE0008F910F900FBE0F901F90189582E084BDA9
:103DF00093E095BD9AEF97BD80936E0008952FB71D
:103E0000F8948091440290914502A0914602B091AD
:103E100047022FBF08952FB7F89460914402709124
:103E2000450280914602909147022FBF0895CF929C
:103E3000DF92EF92FF920F931F932FB7F894409168
:103E400044025091450260914602709147022FBF93
:103E50006A017B01EE24FF248C0120E030E0C016D3
:103E6000D106E206F30610F4415051099A01281BCD
:103E7000390BC9011F910F91FF90EF90DF90CF9008
:103E800008951F920F920FB60F9211248F939F9354
:103E9000AF93BF938091440290914502A091460256
:103EA000B09147020196A11DB11D809344029093E9
:103EB0004502A0934602B0934702BF91AF919F91F4
:103EC0008F910F900FBE0F901F9018950E94A80E13
:103ED000F8942FEF87EA91E6215080409040E1F777
:103EE00000C0000087E090EBDC01809360029093BB
:103EF0006102A0936202B09363029CE088E10FB676
:103F0000F894A895809360000FBE90936000FFCF57
:103F1000E92FF0E093E0EE0FFF1F9A95E1F7E80F2D
:103F2000F11DE855FF4F9491892F8F7092959F70E6
:103F30000895CF93C82FCB010E94881F492F90E08E
:103F4000242F30E054E0220F331F5A95E1F7282B3D
:103F5000392B2038310519F480E090E017C0EC2FA0
:103F6000F0E023E0EE0FFF1F2A95E1F74770E40F22
:103F7000F11D34E0EE0FFF1F3A95E1F7E80FF91F4E
:103F8000EE0FFF1FE050F84985919491CF9108956D
:103F900080E090E00895089580914A0280FF0CC06F
:103FA0008091120190E065E070E00E948427959571
:103FB0008795959587952EC081FF0AC08091120143
:103FC00090E065E070E00E9484279595879522C077
:103FD00082FF08C08091120190E065E070E00E94CD
:103FE000842718C020914B022223D1F03091110177
:103FF000231780F78091120190E065E070E00E9445
:104000008427622F70E00E948427632F70E00E9453
:10401000A127CB018038910530F4009731F0089545
:1040200085E090E008958FE7089581E008958091FC
:104030004A0280FF08C06091100170E07595679595
:104040007595679523C081FF06C06091100170E0EF
:10405000759567951BC082FF04C06091100170E0E8
:1040600012C060914B026623D1F020910F016217BC
:10407000A0F78091100170E090E00E948427622FE9
:1040800070E00E94A1276038710528F46115710560
:1040900021F0862F08958FE7089581E0089561E06B
:1040A00070E0F4CF803F21F40E94CC1F819504C0C2
:1040B000813F29F40E94CC1F80934E020895823FD5
:1040C00021F40E94CC1F819504C0833F29F40E94F3
:1040D000CC1F80934D020895893F19F40E94172048
:1040E00005C08A3F31F40E941720819580934F02CA
:1040F00008958B3F21F40E941720819504C08C3FC6
:1041000029F40E941720809350020895843F21F4DF
:1041100080914C02816017C0853F21F480914C0250
:10412000826011C0863F21F480914C0284600BC0F4
:10413000873F21F480914C02886005C0883F31F4AC
:1041400080914C02806180934C0208958D3F21F450
:1041500080914A0281600BC08E3F21F480914A0217
:10416000826005C08F3F29F480914A028460809369
:104170004A020895803F39F480914E0287FF6CC057
:1041800010924E0269C0813F29F480914E021816A8
:10419000BCF362C090914D02823F29F497FF5CC04E
:1041A00010924D0259C0833F19F41916CCF354C034
:1041B000893F41F480914F0218160CF04DC01092C7
:1041C0004F024AC08A3F29F480914F0287FF44C0C2
:1041D000F6CF8B3F39F48091500287FF3DC010929B
:1041E00050023AC08C3F29F4809150021816BCF35B
:1041F00033C0843F21F480914C028E7F17C0853FED
:1042000021F480914C028D7F11C0863F21F4809172
:104210004C028B7F0BC0873F21F480914C02877F3B
:1042200005C0883F31F480914C028F7E80934C0210
:1042300013C08D3F21F480914A028E7F0BC08E3FC8
:1042400021F480914A028D7F05C08F3F29F480912F
:104250004A028B7F80934A0280914D0281110EC0E9
:1042600080914E0281110AC080914F02811106C0D7
:1042700080915002811102C010924B0208958091EA
:10428000420283FF7EC089E994E00E9497058091F5
:104290004C021F928F9384E994E09F938F930E9426
:1042A000300682E994E00E94970580914D02282F04
:1042B000082E000C330B3F938F938FE894E09F936D
:1042C0008F930E9430068DE894E00E9497058091BC
:1042D0004E02282F082E000C330B3F938F938AE851
:1042E00094E09F938F930E94300688E894E00E94A8
:1042F000970580914F02282F082E000C330B3F9317
:104300008F9385E894E09F938F930E94300683E813
:1043100094E00E94970580915002282F082E000CEF
:10432000330B3F938F9380E894E09F938F930E9489
:1043300030068DE794E00E94970580914B021F9212
:104340008F938AE794E09F938F930E94300688E7CB
:1043500094E00E94970580914A021F928F9385E70F
:1043600094E09F938F930E94300682E794E00E942E
:1043700097058DB79EB74C960FB6F8949EBF0FBEAB
:104380008DBF8CE492E00E94A9110E94FF1E9093C1
:1043900049028093480208951F93CF93DF93809141
:1043A0004802909149020E94171FFC0120914B0284
:1043B000222329F090911301892F90E007C080916A
:1043C000140190E06AE070E00E948427E817F90782
:1043D00008F485C080914D02C0914E02D0914F02E9
:1043E00010915002811107C0C11175C0D11173C065
:1043F000111171C074C02F3F19F02F5F20934B0231
:10440000181624F40E94CC1F80934D0280914D0217
:1044100087FF05C00E94CC1F819580934D021C161A
:1044200024F40E94CC1F80934E0280914E0287FF9D
:1044300005C00E94CC1F819580934E0260914D0271
:10444000662331F1C0914E02CC2311F1062E000CEF
:10445000770B880B990B0E94832623E333E343E316
:104460005FE30E94E7260E944B2660934D026C2F6B
:10447000CC0F770B880B990B0E94832623E333E341
:1044800043E35FE30E94E7260E944B2660934E02BF
:104490001D1624F40E94172080934F0280914F0232
:1044A00087FF05C00E941720819580934F02111647
:1044B00024F40E941720809350028091500287FFBD
:1044C00005C00E941720819580935002DF91CF9103
:1044D0001F910C943F212F3F09F08FCF97CFDF9191
:1044E000CF911F910895ECE4F2E085E0DF011D9289
:1044F0008A95E9F710924B0210924A0208958CEBCC
:1045000096E00E9497051F9281E08F931F9285E0AD
:104510008F938EE696E09F938F930E9430060F90C4
:104520000F900F900F900F900F9008958330E9F146
:1045300028F4813061F0823009F10895853009F462
:1045400062C008F449C0863009F474C008958091AF
:104550001401262F30E0280F311D2F3F310524F4A0
:10456000680F6093140103C08FEF80931401809152
:1045700014011F928F9387EA95E072C08091130116
:10458000262F30E0280F311D2F3F310524F4680F0E
:104590006093130103C08FEF809313018091130187
:1045A0001F928F9385E995E05BC080911201262FC1
:1045B00030E0280F311D2F3F310524F4680F609340
:1045C000120103C08FEF80931201809112011F929C
:1045D0008F9382E895E044C080911101262F30E04E
:1045E000280F311D2F3F310524F4680F609311010E
:1045F00003C08FEF80931101809111011F928F935F
:104600008DE695E02DC080911001262F30E0280F17
:10461000311D2F3F310524F4680F6093100103C052
:104620008FEF80931001809110011F928F9384E58A
:1046300095E016C080910F01262F30E0280F311D24
:104640002F3F310524F4680F60930F0103C08FEFF3
:1046500080930F0180910F011F928F9389E395E062
:104660009F938F930E9430060F900F900F900F90A2
:104670000895833081F128F4813059F08230D1F0EF
:104680000895853009F449C0B8F1863009F456C060
:10469000089580911401681720F4861B80931401FB
:1046A00002C010921401809114011F928F938AE22C
:1046B00095E054C080911301681720F4861B809305
:1046C000130102C010921301809113011F928F9366
:1046D00088E195E043C080911201681720F4861BA1
:1046E0008093120102C010921201809112011F9258
:1046F0008F9385E095E032C080911101681720F416
:10470000861B8093110102C010921101809111014A
:104710001F928F9380EF94E021C080911001681761
:1047200020F4861B8093100102C01092100180912A
:1047300010011F928F9387ED94E010C080910F01BC
:10474000681720F4861B80930F0102C010920F019E
:1047500080910F011F928F938CEB94E09F938F9326
:104760000E9430060F900F900F900F900895CF93F6
:10477000C82F1F928F9381EC97E09F938F930E9495
:10478000300681E090E0A0E0B0E0BC01CD0104C0C3
:10479000660F771F881F991FCA95D2F70E942F1C9A
:1047A0000F900F900F900F90CF910C94ED17CF9327
:1047B000873288F58E3108F00BC18E3009F487C03E
:1047C000D8F4873009F460C08B3009F44FC08630CC
:1047D00009F002C180914202817F8E7F8093420264
:1047E00086EC97E00E94970580E89AE00E94970582
:1047F00081E08093520246C0863109F4B0C020F4B3
:10480000803109F47AC0E8C0893109F491C08B3154
:1048100009F449C0E1C0883349F150F4893209F400
:10482000D5C0853309F4D2C0873209F0D5C0CEC0D7
:10483000833409F4CBC028F48A3308F4CDC08953FB
:10484000C8C0883409F0C8C00E94ED178FE69AE00E
:104850000E9497052FEF83ED90E321508040904018
:10486000E1F700C000000E94661F0CC08DEE97E0CB
:1048700041C086E59AE00E949705809142028160DE
:1048800080934202C1E0ADC080914202C82FC17046
:1048900080FFEFCF82E69AE00E9497058091420266
:1048A000817F8E7F3FC09091420291FBCC27C0F95F
:1048B00081E0C827892FC0FB81F980934202CC2375
:1048C00019F089E49AE029C08BE39AE013C0909133
:1048D000420292FBCC27C0F981E0C827892FC0FB98
:1048E00082F980934202CC2319F08CE29AE015C041
:1048F0008CE19AE00E949705C5CF9091420293FB0C
:10490000CC27C0F981E0C827892FC0FB83F98093A9
:104910004202CC2351F080E19AE00E9497058091F9
:1049200042028160809342025CC083E09AE0E2CF61
:1049300084EF99E00E94970581ED99E00E94970528
:104940008CE899E00E9497058FE599E00E94970511
:104950008AE199E00E9497058BEE98E0CBCF8DED30
:1049600098E00E9497050E9454111F928F9383EC48
:1049700098E09F938F930E94300680910C011F92C4
:104980008F938CEA98E09F938F930E9430068091DA
:104990005F011F928F9389E998E09F938F930E9404
:1049A00030060E940B1F9F938F937F936F9382E833
:1049B00098E09F938F930E9430068DB79EB74296E2
:1049C0000FB6F8949EBF0FBE8DBF5CCF80E001C0D4
:1049D0008D510E94B72356CF80E898E00E9497053A
:1049E000C0E08C2FCF91089580E0089580E0089575
:1049F000CF93C82F80915202813069F020F082302D
:104A000009F449C040C167E08FE00E94E9128823A1
:104A100009F43FC106C067E08FE00E94E9128823D5
:104A200061F08C2F0E94F424811104C08C2F0E940D
:104A3000D7232FC081E090E02CC08C2F0E94F62459
:104A4000811126C0C431E1F070F4CB3081F0C03167
:104A5000D1F40E947F2289EB97E00E94970582E0C3
:104A60008093520215C0C93259F0C83361F486EC04
:104A700097E00E9497058DEB97E00E94970508C08C
:104A80001092520204C187EB97E00E949705FFC085
:104A900081E08170FEC0C43228F5CE3108F0C1C07B
:104AA000CB30A1F1D0F4C73009F0D3C08EE18093B0
:104AB000140182E3809313018AE08093120184E160
:104AC0008093110188E08093100188E280930F01A8
:104AD0008DE596E00E949705BFC0C33149F1C4310E
:104AE000C1F0B7C0CB3409F4A9C028F4C93289F0A9
:104AF000C83361F0AEC0C13509F49EC0C23509F4B7
:104B000099C0CE3409F0A5C06AE09EC00E947F2201
:104B1000A3C080915102882319F0109251029CC0C9
:104B20008AE696E00E94970581E080935202B1C028
:104B300084E496E00E94970582E396E00E94970540
:104B4000809114011F928F938FE296E09F938F9331
:104B50000E9430068DE296E00E9497058BE196E078
:104B60000E949705809113011F928F9388E196E030
:104B70009F938F930E94300686E196E00E949705EE
:104B800087E096E00E949705809112011F928F9313
:104B900084E096E09F938F930E94300682E096E037
:104BA0000E94970581EF95E00E9497058091110181
:104BB0001F928F938EEE95E09F938F930E94300605
:104BC0008CEE95E00E94970587ED95E00E94970591
:104BD000809110011F928F9384ED95E09F938F93A6
:104BE0000E94300682ED95E00E9497058BEB95E0E0
:104BF0000E94970580910F011F928F9388EB95E09B
:104C00009F938F930E94300686EB95E00E94970554
:104C10008DB79EB748960FB6F8949EBF0FBE8DBF56
:104C20001BC0CE51EC2FF0E0E65DFE4F80818093FB
:104C3000510212C061E003C061E006C06AE08091E9
:104C400051020E94962208C0809151020E9439238D
:104C500003C08BE596E013C080915102882369F070
:104C60001F928F9385E596E09F938F930E94300665
:104C70000F900F900F900F9004C082E596E00E9475
:104C8000970581E006C01092520280E002C080E0E9
:104C900000CFCF9108950E9452266894B1110C94D0
:104CA000E12608950E94C62688F09F5798F0B92FF4
:104CB0009927B751B0F0E1F0660F771F881F991F51
:104CC0001AF0BA95C9F714C0B13091F00E94E026ED
:104CD000B1E008950C94E026672F782F8827B85FFD
:104CE00039F0B93FCCF3869577956795B395D9F7A9
:104CF0003EF490958095709561957F4F8F4F9F4FB3
:104D00000895E89409C097FB3EF4909580957095BE
:104D100061957F4F8F4F9F4F9923A9F0F92F96E907
:104D2000BB279395F695879577956795B795F1117C
:104D3000F8CFFAF4BB0F11F460FF1BC06F5F7F4F19
:104D40008F4F9F4F16C0882311F096E911C077232B
:104D500021F09EE8872F762F05C0662371F096E834
:104D6000862F70E060E02AF09A95660F771F881F03
:104D7000DAF7880F9695879597F9089557FD90581B
:104D8000440F551F59F05F3F71F04795880F97FB0F
:104D9000991F61F09F3F79F08795089512161306C9
:104DA0001406551FF2CF4695F1DF08C016161706F8
:104DB0001806991FF1CF869571056105089408952D
:104DC000E894BB2766277727CB0197F908950E94BF
:104DD000F9260C9473270E94652738F00E946C27EF
:104DE00020F0952311F00C945C270C9462270C940E
:104DF000E1260E94BE2678F39923C9F35523B9F31F
:104E0000950F50E0551FAA27EE27FF27BB27002448
:104E10000894679520F4E20FF31FB41F0A1E220FB7
:104E2000331F441FAA1F6695A9F7779530F4F30F37
:104E3000B41F0A1E121E08F46395330F441FAA1FE5
:104E4000221F769599F7879520F4B40F0A1E121E3B
:104E5000631F440FAA1F221F331F8695A9F7862FB1
:104E6000712D602D11249F5750409AF0F1F0882346
:104E70004AF0EE0FFF1FBB1F661F771F881F915060
:104E80005040A9F79E3F510580F00C945C270C948C
:104E9000E1265F3FE4F3983ED4F3869577956795D6
:104EA000B795F795E7959F5FC1F7FE2B880F911D8A
:104EB0009695879597F9089597F99F6780E870E030
:104EC00060E008959FEF80EC089500240A94161680
:104ED000170618060906089500240A9412161306E8
:104EE000140605060895092E0394000C11F4882376
:104EF00052F0BB0F40F4BF2B11F460FF04C06F5F92
:104F00007F4F8F4F9F4F08950024552704C0080EF0
:104F1000591F880F991F009729F076956795B8F368
:104F20007105B9F7802D952F0895991B79E004C07C
:104F3000991F961708F0961B881F7A95C9F78095D8
:104F4000089597FB072E16F4009407D077FD09D03B
:104F50000E94BB2707FC05D03EF4909581959F4F9A
:104F60000895709561957F4F0895EE0FFF1F05908E
:104F7000F491E02D0994AA1BBB1B51E107C0AA1FA5
:104F8000BB1FA617B70710F0A61BB70B881F991FEA
:104F90005A95A9F780959095BC01CD010895F89494
:024FA000FFCF41
:104FA200FFFF130A040BE10AAD0A790A013802284D
:104FB20008140A321E404D3622DA038D0357033598
:104FC20003C102DA02F3020C030001020304050624
:044FD20007080900C3
:106800000000EA44E944E2440400050006000700F1
:10681000080009000A000B000C000D000E000F001C
:1068200010001100120013001400150016001700CC
:10683000180019001A001B001C001D001E001F007C
:10684000200021002200230024002500260027002C
:10685000280029002A002B002C002D002E002F00DC
:10686000300031A132003300340035A1360037004A
:10687000380082003A003B003C003D003E003F00F3
:1068800040004100420043004400450046004700EC
:10689000480049004A004B004C004D004E004F009C
:1068A000500051005200530067005400550056003C
:1068B000580059005A005B005C005D005E005F00FC
:1068C0006000610062006300640000005700000087
:1068D000CD440000000000000000000000000000A7
:1068E0000000000000006620000000000000000022
:1068F000E000E100E200E300E400E500E600E7007C
:106900000100010001000100EA4401000100E2442D
:106910000100010001000100460001004A004B0097
:10692000010001004700480001000100E9440100A6
:106930000100010001000100010001003A003B00DC
:106940003C003D003E003F0040004100420043004B
:10695000010001004C00010001004400450052000C
:1069600049000100010050004F0001004D004E00A1
:1069700051000100010001000100010001000100BF
:1069800001000100010001000100010001000100FF
:1069900001000100010001000100010001004D00A3
:1069A0004A004E004B0001000100010001000100FF
:1069B00001000100010001000100010001000100CF
:1069C00001000100010001000100010001000100BF
:1069D00001000100010001000100010001000100AF
:1069E000010001000100010001000100010001009F
:1069F000010001000100010001000100010001008F
:00000001FF
